:1000000042C1189518951895189518951895189532
:10001000189518951895CCC0189518951895189599
:100020001895189518950100890008006F00740054
:10003000770079007C008000820085000100A90023
:1000400008008F009400970099009C00A000A20077
:10005000A5000100C9000800AF00B400B700B90056
:10006000BC00C000C200C5000600A000000002E005
:100070000BB908E90AB900B5006800BD06E800BD83
:1000800000B50F7700BD0CE009B900E000BD0FEF2F
:1000900007BB04BB0EEF01BB00E002BB0093A20054
:1000A0000093A000089502E010E012BF15E013BF16
:1000B00028B720FFFDCF18B7116018BF0A95A1F728
:1000C000089553D1902F112311F4822F02C089E09B
:1000D000821B9923F1F4082FE6E2F0E0F1C0C0980A
:1000E000C19AC298C39A15C0C098C198FACFC09A55
:1000F000FCCFC09AC1980BC0C09AC198C29A08C0E0
:10010000C098FBCFC098C19AF9CFC098C19AC29845
:10011000C3989130F1F4082FECE3F0E0D1C0A89837
:10012000A99AAA98AB9A15C0A898A998FACFA89AA4
:10013000FCCFA89AA9980BC0A89AA998AA9A08C017
:10014000A898FBCFA898A99AF9CFA898A99AAA9895
:10015000AB989230F1F4082FE2E5F0E0B1C094984A
:10016000959A9698979A15C094989598FACF949ADC
:10017000FCCF949A95980BC0949A9598969A08C03B
:100180009498FBCF9498959AF9CF9498959A9698CD
:10019000979880E002C087DF83950091A3008017C5
:1001A000D0F381DF00E818B3102718BBE2E0E0C00D
:1001B000FA93EA932A931A930A932FB7E0EAF0E0AE
:1001C0000281002331F51CB106E000000A95E9F731
:1001D0001CB95E9BFECF5E9A17FBD6F416FB16F495
:1001E00001E001C000E00083012F007311F400E082
:1001F0000BC0012F0073003111F401E005C0012F85
:100200000073003211F402E001831F70138301C0F8
:1002100012832FBF099119912991E991F9911895AC
:10022000A2D0A4EAB0E000E0E4EAF0E001831FDF3E
:10023000789426C02C911091A0000091A10041DF7C
:100240000C9103950C93093010F001E00C93E2EA55
:10025000F0E000810A95008301E0E4EAF0E0018328
:100260000091A200002331F7E4EAF0E001810023CD
:1002700039F000E001830CE00CB95E9BFECF5E9A82
:1002800001E00C93EDCF0FE90DBF00E00EBFC0E819
:10029000D0E077D0002309F084D0C2DF9CD09BC08F
:1002A0005FD0702D5DD0602D5BD0502D59D0402D8A
:1002B00057D0102C01FA54D0202C52D0302C089555
:1002C000F5DF041B10E003C0EFDF041B150B20E07B
:1002D00030E005C0E5DF041B150B260B370BE0F003
:1002E00010FC1DC03DD0402D3BD0E00FF11F041786
:1002F000100540E02407340778F446F4C895002D33
:100300000024E22DF32DE01BF0090994E00FF11F0A
:1003100027D0202C25D0302CE22DF32D099411F478
:10032000BEF7ECCF31960EF0319650E060E070E011
:1003300017D0402D4B3F68F079F34F3F41F04E3FCF
:1003400021F00ED0702D0CD0602D0AD0502D08D089
:10035000402D041B150B260B370B11F3E8F2E2CFEF
:10036000C89531960895BA93AA939A938A9308955B
:1003700099818881F0E00FB6F894CE0FDF1F0FBE91
:10038000089501E0089520E002D0E9F708952D9343
:1003900001501040202F212B08952591F8DFE9F717
:1003A000089588E690E0FC0105911491FC013296D5
:1003B000A591B491FC01349625913491422F432BA1
:1003C00019F0F901EADF01C0DEDF069610E08E3693
:0C03D000910748F3089500008895FECFC7
:00000001FF
